:02000000DF28F7
:08000800DF00030E8312A000CB
:0E0010000A0EA100040EA2008A110A12E528B1
:10002000AE08031D14280800F930FF3E031D1528F3
:10003000AE0B14280800FA30AE001020FA30AE00E3
:100040001020FA30AE001020FA30AE001020AD0BB8
:100050001B280800AB0B2D28080000000000000042
:100060000000000000000000AB0B2D2808008312E8
:100070009F149F1839281E08AD00080037202D0A4C
:10008000A6000130260203180800FF30A600080071
:100090000D309F00083083169F00073083129900AF
:1000A000DA30831685000230950081130230960005
:1000B000C83083128B0030309000AC08031D05154A
:1000C000FF30AE001020FF30AE0010200511851665
:1000D0000330AD001B203E20A301A40108008312C1
:1000E0000515C830AE0010200511C830AE00102034
:1000F0000515C830AE0010200511850185120508D0
:10010000AB000B108B1563008B110130AC00482045
:10011000080001308312AC004820A801A901053075
:100120002902031D9528FF3028020318D3288518BB
:10013000A02805153230AE001020851C9D286F20A8
:1001400037202D08A50026020318CF28A301A401FB
:100150003230AE0010203E20AA0104302A020318DB
:10016000CE2885308F00ED308E000C1010140C1846
:10017000CB2837202D08A50026020318B728051420
:1001800005150530AB002A2005109630AE00102072
:100190000511FF30AA001010AA0AAD280511A80AFF
:1001A0000319A90A8F28A30A0319A40A2408513C99
:1001B000031DDC282308403C031C6F208D2883127C
:1001C0002710A7108A110A12892883120B1CEB280A
:1001D0000508AF000B10220E8400210E8A00200EAD
:0801E0008300DF0E5F0E090031
:02400E00041E8E
:00000001FF
